:020000040000FA
:040000006A303A2800
:08000800A000030EA100831209
:100010008B1C32288B1031181428B11C3228643004
:10002000010203183128182800001628172818285C
:1000300019281A281B281C281D281E281F283110A3
:10004000B114A810031005190314AA0DA90DA80DC9
:10005000B00B322831152A08AF002908AE00280855
:10006000AD00B11081010B11210E8300A00E200EF6
:02007000090085
:0C007400203084008001840A80300402E7
:10008000031C3C281230B000512283160C30850529
:1000900087018312850187010730990000309A009B
:1000A000103083168E008312603083168F00831207
:1000B0000030831691009F008312C83083168100A0
:1000C000831231309000003083168C008312103080
:1000D0008B00BC1B7128851971286400851D6D2853
:1000E00082233C1C74280C2381018E018F010B118B
:1000F0008B100B108C018B178C203119A2202E2213
:10010000B30B8A28031085190314B90DF030390296
:100110000319BD2121237C286400311808000B1D20
:1001200008000B11B11031141230B000051D9D28CC
:10013000321483160113831208003210831601173C
:100140008312080031110130B7008B1320303707BC
:1001500083169B001C141A088312A400A500C0304B
:10016000A5061030370783169B001C141A0883124B
:10017000A3000030370783169B001C141A08831253
:10018000A2008B17321CCA2822090339A200A30936
:10019000A409A50922082D02031DB72923082E0250
:1001A000031DB72924082F02031D442901303702FB
:1001B000031DE1283C19E0283D18E1283D143E14B8
:1001C000762202303702031DEC283C19EB28BD18BB
:1001D000EC28BD143E147D2203303702031DF7289E
:1001E0003C19F6283D19F7283D153E1484220430A9
:1001F0003702031D02293C190129BD190229BD1529
:100200003E148B2205303702031D0D293C190C29A1
:100210003D1A0D293D163E14922206303702031D69
:1002200018293C191729BD1A1829BD163E14992200
:1002300007303702031D23293C1922293D1B23299E
:100240003D173E14A02208303702031D2E293C1909
:100250002D29BD1B2E29BD173E14A72209303702B8
:10026000031D39293C1938294218392942143E14F2
:10027000AE220A303702031D44293C194329C21813
:100280004429C2143E14B52225082F02031DB729A4
:1002900001303702031D53293C1952293D1C5329B3
:1002A0003D103E14BC2202303702031D5E293C196A
:1002B0005D29BD1C5E29BD103E14C02203303702EB
:1002C000031D69293C1968293D1D69293D113E140A
:1002D000C42204303702031D74293C197329BD1D43
:1002E0007429BD113E14C82205303702031D7F2931
:1002F0003C197E293D1E7F293D123E14CC2206303A
:100300003702031D8A293C198929BD1E8A29BD127D
:100310003E14D02207303702031D95293C19942939
:100320003D1F95293D133E14D42208303702031D8A
:10033000A0293C199F29BD1FA029BD133E14D82216
:1003400009303702031DAB293C19AA29421CAB29ED
:1003500042103E14DC220A303702031DB6293C1934
:10036000B529C21CB629C2103E14E022B729B70A2B
:100370000B30370203180800A5280130B600B3007F
:10038000B400B500B70085018701B1138C20B30B11
:10039000FD29031085190314B90DF0303902031932
:1003A000242AB40BFD29013037020319E42202305C
:1003B00037020319E822033037020319EC22043014
:1003C00037020319F022053037020319F4220630F0
:1003D00037020319F822073037020319FC220830CC
:1003E00037020319002309303702031904230A30A6
:1003F0003702031908239630B400311DC629311184
:10040000321C072A2D090339AD00AE09AF092F1C94
:10041000B1132F1CC629B11BC6292E18C629B11726
:100420008B1320303707BB002F08BA003C22103056
:100430003707BB002E08BA003C2200303707BB004C
:100440002D08BA003C228B1785018701B70AB60137
:100450000B303702031CC6290C2308003E1C080081
:100460003E101030BB003D08BA003C223030BB00CB
:100470004208BA003C2208008B133A0883161C1568
:100480009A0083123B0883169B0055309D00AA30CA
:100490009D009C1464009C184A2A1C1183128B171F
:1004A0000800831600309B001C141A088312BC003D
:1004B000831610309B001C141A0883123C18BD00D0
:1004C000831630309B001C141A0883123C18C2009B
:1004D000831620309B001C141A088312C1000130BF
:1004E000C11BC100C1080319C1000800051640085E
:1004F0004107D0000F08D1000800851640084107C9
:10050000D2000F08D3000800051440084107D400AA
:100510000F08D5000800851440084107D6000F08D1
:10052000D7000800871440084107D8000F08D900F9
:100530000800071540084107DA000F08DB00080033
:10054000071440084107DC000F08DD00080087168B
:1005500040084107DE000F08DF00080007164008CA
:100560004107CC000F08CD0008008715400841075F
:10057000CE000F08CF00080005128E018F01080081
:1005800085128E018F01080005108E018F01080071
:1005900085108E018F01080087108E018F010800E1
:1005A00007118E018F01080007108E018F010800CE
:1005B00087128E018F01080007128E018F0108003B
:1005C00087118E018F0108000508103A8500080088
:1005D0000508203A850008000508013A8500080052
:1005E0000508023A850008000708023A870008005B
:1005F0000708043A870008000708013A8700080046
:100600000708203A870008000708103A870008000A
:100610000708083A870008003D180516BD1885161A
:100620003D190514BD1985143D1A8714BD1A071507
:100630003D1B0714BD1B871642180716C2188715E5
:1006400008003C1D080050084002031D2C2B5108D7
:100650000F02031C2C2B051252084002031D352BE0
:1006600053080F02031C352B851254084002031D4A
:100670003E2B55080F02031C3E2B05105608400266
:10068000031D472B57080F02031C472B85105808E2
:100690004002031D502B59080F02031C502B8710DA
:1006A0005A084002031D592B5B080F02031C592BEB
:1006B00007115C084002031D622B5D080F02031C3A
:1006C000622B07105E084002031D6B2B5F080F02B0
:1006D000031C6B2B87124C084002031D742B4D0822
:1006E0000F02031C742B07124E084002031D7D2BC2
:1006F0004F080F02031C7D2B87110C1C08000C10E7
:10070000C00A0800B601B301B4013C1C8A2BBC012D
:10071000BC14912BBC1C8F2BBC013C15912BBC0134
:100720003C143C08B6006400952B962B972B982B15
:10073000992BB41B0516B41F0512B30B932BB40BE6
:10074000932B0310B60CB608031D932B0030BB008F
:080750003C08BA003C2208003D
:084000000900030006000600A0
:02400E00CC33B1
:10420000010003000300030003000200020002009B
:1042100002000000000000000000FF00FF00FF009F
:10422000000000000000000000000000000000008E
:104230000000C000C000C000C000FF00FF00FF0081
:104240000100C300F300CF00FF00C300F300CF0064
:10425000FF00C300F300CF00FF00FF00FF00FF00DE
:104260000000FF00FF00FF00FF00FF00FF00FF0055
:10427000FF00FF00FF00FF00FF00FF00FF00FF0046
:10428000FF00FF00FF00FF00FF00FF00FF00FF0036
:10429000FF00FF00FF00FF00FF00FF00FF00FF0026
:1042A000FF00FF00FF00FF00FF00FF00FF00FF0016
:1042B000FF00FF00FF00FF00FF00FF00FF00FF0006
:1042C000FF00FF00FF00FF00FF00FF00FF00FF00F6
:1042D000FF00FF00FF00FF00FF00FF00FF00FF00E6
:1042E000FF00FF00FF00FF00FF00FF00FF00FF00D6
:1042F000FF00FF00FF00FF00FF00FF00FF00AA001B
:00000001FF
